:100000000C9461000C947E000C947E000C947E0095
:100010000C947E000C947E000C947E000C947E0068
:100020000C947E000C947E000C947E000C947E0058
:100030000C947E000C947E000C947E000C947E0048
:100040000C945A010C947E000C947E000C947E005B
:100050000C947E000C947E000C947E000C947E0028
:100060000C947E000C947E00000000002400270009
:100070002A0000000000250028002B0000000000DE
:1000800023002600290004040404040404040202DA
:100090000202020203030303030301020408102007
:1000A0004080010204081020010204081020000012
:1000B0000008000201000003040700000000000027
:1000C000000011241FBECFEFD8E0DEBFCDBF13E08C
:1000D000A0E0B1E0ECE7F9E002C005900D92A43B8E
:1000E000B107D9F723E0A4EBB3E001C01D92AD3C0A
:1000F000B207E1F70E94A4010C94BC040C94000028
:10010000833081F028F4813099F08230A9F008958D
:100110008730A9F08830C9F08430B1F48091800034
:100120008F7D03C0809180008F7780938000089539
:1001300084B58F7784BD089584B58F7DFBCF809182
:10014000B0008F778093B00008958091B0008F7DCC
:10015000F9CFCF93DF93282F30E0F901E255FF4F1D
:100160008491F901E656FF4FD491F901EA57FF4F08
:10017000C491CC23A1F081110E948000EC2FF0E00B
:10018000EE0FFF1FE458FF4FA591B491EC91ED23C2
:1001900081E090E009F480E0DF91CF91089580E064
:1001A00090E0FACF1F93CF93DF93282F30E0F9012F
:1001B000E255FF4F8491F901E656FF4FD491F901C2
:1001C000EA57FF4FC491CC23A9F0162F81110E944A
:1001D0008000EC2FF0E0EE0FFF1FEE58FF4FA591CF
:1001E000B4918FB7F894EC91111108C0D095DE232B
:1001F000DC938FBFDF91CF911F910895DE2BF8CF55
:10020000CF93DF9390E0FC01E656FF4F24918A578D
:100210009F4FFC0184918823C9F090E0880F991FBB
:10022000FC01E859FF4FA591B491FC01EE58FF4F36
:10023000C591D49161110DC09FB7F8948C91209510
:1002400082238C938881282328839FBFDF91CF91BD
:100250000895623051F49FB7F8943C91822F8095B5
:1002600083238C93E8812E2BEFCF8FB7F894EC91FA
:100270002E2B2C938FBFEACF8E50806480937C000E
:1002800080917A00806480937A0080917A0086FD64
:10029000FCCF809178009091790008952FB7F89461
:1002A0006091C9037091CA038091CB039091CC03F4
:1002B0002FBF08951F920F920FB60F9211242F9304
:1002C0003F938F939F93AF93BF938091C903909176
:1002D000CA03A091CB03B091CC033091C80323E0B3
:1002E000230F2D3758F50196A11DB11D2093C8038A
:1002F0008093C9039093CA03A093CB03B093CC031C
:100300008091C4039091C503A091C603B091C70327
:100310000196A11DB11D8093C4039093C503A093C2
:10032000C603B093C703BF91AF919F918F913F9147
:100330002F910F900FBE0F901F90189526E8230F56
:100340000296A11DB11DD2CF789484B5826084BD80
:1003500084B5816084BD85B5826085BD85B58160C9
:1003600085BD80916E00816080936E001092810047
:100370008091810082608093810080918100816002
:1003800080938100809180008160809380008091C3
:10039000B10084608093B1008091B000816080934F
:1003A000B00080917A00846080937A0080917A0016
:1003B000826080937A0080917A00816080937A00D5
:1003C00080917A00806880937A001092C10060E08A
:1003D00081E10E94000162E084E00E94000161E08E
:1003E0008BE00E94000161E083E00E94000160E078
:1003F00089E00E94000160E08EE00E94000160E060
:100400008BE00E94D200CC24CA94A3E0DA2EE12C27
:10041000F12CB4E64B2E512C612C712C2224239408
:1004200080E10E943C018C0181E0011522E012076D
:100430000CF480E08093C3038091C2038823A1F071
:10044000011582E018070CF458C10E944E01683E65
:1004500073408105910540F060E083E00E94D20086
:100460001092C2031092C1038EE00E943C01EC0185
:1004700083E10E943C012596C80FD91FCF3FD3408E
:100480000CF0FAC08EE00E943C01EC0183E10E9476
:100490003C012596C80FD91FBE01DD0F880B990BB3
:1004A000011522E012070CF4EAC0F4E0660F771F92
:1004B000881F991FFA95D1F7A70196010E942A0477
:1004C000E9018FE00E943C01AA24AA9463E0B62EC1
:1004D0008A3F93402CF48FE00E943C0105965C011A
:1004E00089E00E94A900332433948130910509F0FA
:1004F000312C019709F056C08091C003811152C080
:100500008091C10381114EC024E630E0D5010E94E4
:10051000A104A70196010E942A0449015A01809171
:10052000BE039091BF03011512400CF4B0C044E02B
:10053000CC0FDD1F4A95E1F7C80FD91FCC0FDD1F87
:10054000CC56DE4F888199810197F9F40E94D2033D
:10055000A30192010E942A04681579058A059B056A
:10056000A4F461E08BE00E94D20061E083E00E948D
:10057000D2000E944E016093BA037093BB03809334
:10058000BC039093BD032092B9038091BE03909168
:10059000BF03019660E170E00E948D049093BF0359
:1005A0008093BE0381E10E94A9008C0184E00E9437
:1005B000A900EC010130110511F0892B59F580914A
:1005C000B803811121C00E944E018090B403909025
:1005D000B503A090B603B090B703681979098A09EA
:1005E0009B09633371058105910570F00E944E01EE
:1005F0006093B4037093B5038093B6039093B703ED
:100600001092BF031092BE0381E00130110519F072
:10061000CD2B09F080E08093B8033092C003809125
:10062000B903882309F10E944E010091BA03109189
:10063000BB032091BC033091BD03601B710B820B87
:10064000930B6A3071058105910570F060E08BE0D5
:100650000E94D2008091C103811104C060E083E058
:100660000E94D2001092B90380E090E0892B09F437
:10067000D7CE0E940000D4CECFEFD3E00DCFE3E081
:10068000660F771F881F991FEA95D1F715CF23E0D2
:10069000CC0FDD1F2A95E1F7C80FD91FCC0FDD1F46
:1006A000CC5FDE4F888199810197F9F40E94D203D3
:1006B000A30192010E942A04681579058A059B0509
:1006C000A4F461E08BE00E94D20061E083E00E942C
:1006D000D2000E944E016093BA037093BB038093D3
:1006E000BC039093BD032092B9038091BE03909107
:1006F000BF03019668E070E04FCF0E944E01643F57
:1007000071408105910508F4AFCEA6CE8F929F92DD
:10071000AF92BF92CF92DF92EF92FF92CF93DF938F
:10072000EC01688179818A819B8161157105810560
:10073000910521F464E279ED8BE597E02DE133EF4B
:1007400041E050E00E942A0449015A019B01AC019A
:10075000A7EAB1E40E9449046B017C01ACEEB4EF5E
:10076000A50194010E945704C60ED71EE81EF91E6B
:10077000F7FE06C081E0C81AD108E10880E8F80A4F
:10078000C882D982EA82FB82C701B6019F77DF91D6
:10079000CF91FF90EF90DF90CF90BF90AF909F9060
:1007A0008F9008958F929F92AF92BF92CF92DF92D7
:1007B000EF92FF926091000170910101809102011E
:1007C00090910301611571058105910521F464E2A1
:1007D00079ED8BE597E02DE133EF41E050E00E94A9
:1007E0002A0449015A019B01AC01A7EAB1E40E9425
:1007F00049046B017C01ACEEB4EFA50194010E94A9
:100800005704C60ED71EE81EF91EF7FE06C081E08B
:10081000C81AD108E10880E8F80AC0920001D09215
:100820000101E0920201F0920301C701B6019F7736
:10083000FF90EF90DF90CF90BF90AF909F908F9000
:1008400008956093000170930101809302019093D9
:1008500003010895052E97FB1EF400940E944104A5
:1008600057FD07D00E945C0407FC03D04EF40C94A3
:10087000410450954095309521953F4F4F4F5F4F24
:10088000089590958095709561957F4F8F4F9F4FFC
:1008900008950E947E04A59F900DB49F900DA49F83
:1008A000800D911D11240895B7FF0C9449040E94F6
:1008B0004904821B930B0895A1E21A2EAA1BBB1BAD
:1008C000FD010DC0AA1FBB1FEE1FFF1FA217B3071C
:1008D000E407F50720F0A21BB30BE40BF50B661F32
:1008E000771F881F991F1A9469F7609570958095F6
:1008F00090959B01AC01BD01CF010895A29FB0016D
:10090000B39FC001A39F700D811D1124911DB29F43
:10091000700D811D1124911D089597FB072E16F46B
:10092000009407D077FD09D00E94A80407FC05D0E9
:100930003EF4909581959F4F0895709561957F4FF6
:1009400008950E947E04B7FF0895821B930B0895BB
:10095000AA1BBB1B51E107C0AA1FBB1FA617B707E5
:1009600010F0A61BB70B881F991F5A95A9F7809501
:0C0970009095BC01CD010895F894FFCFD4
:10097C00010000000000000000000000000000006A
:10098C00000000000100000000000000000000005A
:10099C000000000001000000000000000100000049
:1009AC000000000001000000010000000000010038
:1009BC000000000001000000010000000100000028
:1009CC000100000001000100000001000100000016
:1009DC000100000001000100010000000100010005
:1009EC0001000000010001000100010001000100F4
:1009FC0001000000010001000100010001000100E4
:100A0C0001000100000000000000000000000000D8
:100A1C0000000000000000000000000000000000CA
:100A2C0000000000010000000000000000000000B9
:100A3C0000000000000000000000000000000000AA
:100A4C000000000001000000000000000000000099
:100A5C000000000001000000000000000000000089
:100A6C000000000001000000000000000000010078
:100A7C000000000000000000010000000000000069
:100A8C000000000001000000000000000100000058
:100A9C000000000001000000000000000100000048
:100AAC000000000001000000000001000000000038
:100ABC000100000000000100000000000100000027
:100ACC000000000001000000010000000000010017
:100ADC000000000001000000010000000000010007
:100AEC0000000000010000000100000001000000F7
:100AFC0001000000000001000000010000000100E6
:100B0C0000000000010000000100000001000000D6
:100B1C0001000000010000000100000001000000C5
:100B2C0001000000010001000000010000000100B4
:100B3C0000000100010000000100000001000000A5
:100B4C000100000001000100000001000100000094
:100B5C000100000001000100000001000100000084
:100B6C000100000001000100010000000100010073
:100B7C000000010001000000010001000000010064
:100B8C000100000001000100010000000100010053
:100B9C000100000001000100010000000100010043
:100BAC000100000001000100010001000100000033
:100BBC000100010001000100000001000100010022
:100BCC000100000001000100010001000100010012
:100BDC000100000001000100010001000100010002
:100BEC0001000000010001000100010001000100F2
:100BFC0001000100010001000100010001000100E1
:100C0C0001000000010001000100010001000100D1
:100C1C0001000100010001000100010001000100C0
:040C2C0001000100C2
:00000001FF
